:020000040000FA
:10000000831204309908031D49280730990083168C
:100010008113133095009F01DB308500FF23900092
:1000200083122030850005305E2033200508A000B3
:10003000043085002408201A250859202030850026
:1000400085192C2826085920043085002408201AF8
:10005000250859202030850020080339273E8400D8
:1000600000085E20162883162430840000309B0090
:100070001C141A0880009B0A840A04082D3A031DE8
:10008000382883122C082B06013E03190800033080
:100090004928AC002C08AB000430850002305E20FB
:1000A0002030850003305E20AB0B4C280A305E20E8
:1000B0004A28A2006420A20B5A280800A30064303A
:1000C0005920A30B5F280800C6300000FF3E031D27
:0A00D0006528000000000000080091
:02400E00843FED
:104200001E006400AF000A0014001E002800A90070
:02421000560056
:104220004C004500440020005300740072006F00F1
:104230006200650020005200650076002E0020001C
:104240004600200068007400740070003A002F00DF
:104250002F00700069006300700072006F006A0038
:1042600065006300740073002E006F007200670029
:084270002E0075006B00200018
:00000001FF
